:020000040000FA
:06000000713001303A28C6
:08000800A000030EA100831209
:100010008B1C32288B1031181428B11C3228643004
:10002000010203183128182800001628172818285C
:1000300019281A281B281C281D281E281F283110A3
:10004000B114A810031005190314AA0DA90DA80DC9
:10005000B00B322831152A08AF002908AE00280855
:10006000AD00B11081010B11210E8300A00E200EF6
:02007000090085
:0C007400203084008001840A80300402E7
:10008000031C3C281230B000662183160C30850515
:1000900087018312850187010730990000309A009B
:1000A000103083168E008312603083168F00831207
:1000B0000030831691009F008312C83083168100A0
:1000C000831231309000003083168C008312103080
:1000D0008B00BC1B7128851971286400851D6D2853
:1000E000C421C12181018E018F010B118B100B10D6
:1000F0008C018B178A203119A0204821B30B882846
:10010000031085190314B90DF03039020319F120D9
:10011000EE217A286400311808000B1D08000B112D
:10012000B11031141230B000051D9B283214831613
:10013000011383120800321083160117831208007E
:1001400031110130B7008B132030370783169B0025
:100150001C141A088312A400A500C030A506103094
:10016000370783169B001C141A088312A300003063
:10017000370783169B001C141A088312A2008B17E2
:10018000321CC82822090339A200A309A409A50921
:1001900022082D02031DEB2823082E02031DEB2845
:1001A00024082F02031DDD2801303702031DDD283E
:1001B0003D18DD283D143E149D2125082F02031D06
:1001C000EB2801303702031DEA283D1CEA283D10C8
:1001D0003E14A721EB28B70A0230370203180800A3
:1001E000A3280130B600B300B400B500B700850104
:1001F0008701B113B7218A20B30B16290310851983
:100200000314B90DF030390203193D29B41F8501DB
:10021000B41F8701B40B1629B50B16290230B5009F
:10022000013037020319AE219630B400311DFB288E
:100230003111321C20292D090339AD00AE09AF0957
:100240002F1CB1132F1CFB28B11BFB282E18FB28D9
:10025000B1178B1320303707BB002F08BA0051218C
:1002600010303707BB002E08BA0051210030370785
:10027000BB002D08BA0051218B17BE2185018701D3
:10028000B70AB60102303702031CFB28C12108005F
:100290003E1C08003E101030BB003D08BA00512142
:1002A00008008B133A0883161C159A0083123B082A
:1002B00083169B0055309D00AA309D009C1464005D
:1002C0009C185F291C1183128B17080083160030BD
:1002D0009B001C141A088312BC00831610309B006C
:1002E0001C141A088312BD00831620309B001C14B6
:1002F0001A088312C3000130C3080319C300831610
:1003000030309B001C141A088312C4004430D500FE
:10031000831670309B001C141A088312D6000E0737
:10032000D70057075507D8007030BB005708BA00F0
:1003300051210230C100C20008000130BD0001306F
:10034000C100C200C8005414D41054110800013078
:10035000C100C2005410D4105415080038093339B4
:100360008500B8003F093F398700BF000800113001
:100370008500B80013308700BF000800B801BF0136
:1003800008003D189D210800B601B301B4013C1CD2
:10039000CC29BC01BC14CE29BC013C143C08B600DD
:1003A0006400D229D329D429D529D629FF30B41BFA
:1003B0008500B41B8700B41F8501B41F8701B30BF0
:1003C000D029B40BD0290310B60CB608031DD029D0
:1003D0000030BB003C08BA0051210800D4080319C2
:1003E0002E2307305405031908008F08031908004D
:1003F0008F0178308E005D095B05CA005E095C05DF
:10040000CB005B095D05CC005C095E05CD00C8082A
:100410000319102AFF303C1CC800C80FCB2A5323F5
:10042000C20B08006430C200C10B08004308C100C1
:100430000130C800C9002E23551C222A571C5B140A
:10044000D71C5B10551D282A571DDB14D71DDB1048
:10045000D51D2E2A571E5B15D71E5B11551E342A3B
:10046000571FDB15D71FDB11D51E3A2A581C5B1608
:10047000D81C5B12551F402A581DDB16D81DDB12F5
:10048000D51F462A581E5B17D81E5B13561C4C2AD4
:10049000581FDB17D81FDB13D61C522A561F5C14BB
:1004A000D61F5C105418DC14D418DC145419DC105A
:1004B000541D5E2ACE0B5E2ADB01DB01C5015B18F1
:1004C000C50ADB18C50A5B19C50ADB19C50A5B1A20
:1004D000C50ADB1AC50A5B1BC50ADB1BC50A5C180B
:1004E000C50AC6015D18C60ADD18C60A5D19C60A26
:1004F000DD19C60A5D1AC60ADD1AC60A5D1BC60AE0
:10050000DD1BC60A5E18C60AC7015B085D06C0008F
:100510004018C70AC018C70A4019C70AC019C70A35
:10052000401AC70AC01AC70A401BC70AC01BC70A1D
:100530005C085E06C0004018C70AC018C70AC70B8F
:10054000C02A5418A82AD418B42A5419B92A080061
:10055000440845020318B12A46084502031CC02A74
:1005600008005410D414080044084502031CC02A93
:10057000080045084602031CC02A1430CE000800BB
:100580005D08DB005E08DC005419DC105418DC1434
:10059000D418DC1408004808C9004A180516CA18FF
:1005A00085164A190514CA1985144A1A8714CA1AD5
:1005B00007154A1B0714CA1B87164B180716CB18BA
:1005C000871549080E020318FD2A4C180512CC188D
:1005D00085124C190510CC1985104C1A8710CC1AAD
:1005E00007114C1B0710CC1B87124D180712CD1892
:1005F0008711FF304802031908008F08031D080007
:100600008A2049080E02031CFD2A4A180512CA183E
:1006100085124A190510CA1985104A1A8710CA1A74
:1006200007114A1B0710CA1B87124B180712CB1859
:1006300087114C180516CC1885164C190514CC19C1
:1006400085144C1A8714CC1A07154C1B0714CC1BA5
:1006500087164D180716CD18871508005508DF00B6
:100660004123D5005608DF004123D6005708DF009C
:10067000551C4123D7005808DF00D51C4123D80062
:100680000800C001DF080319DF035F184014DF1AF8
:1006900040144008C0015F1C4014DF1E4014C00518
:1006A000C00C5F0C08004A180516CA1885164A19AE
:1006B0000514CA1985144A1A8714CA1A07154A1B41
:1006C0000714CA1B87164B180716CB188715CA01C3
:1006D000CB014C180512CC1885124C190510CC19F9
:1006E00085104C1A8710CC1A07114C1B0710CC1B15
:1006F00087124D180712CD188711CC01CD015B0868
:10070000DD005C08DE00DB08031D0800DC08031DBB
:060710000800541108006E
:084000000E000300060007009A
:02400E00CC33B1
:10420000010003000300030003000200020002009B
:1042100002000000000000000000FF00FF00FF009F
:10422000000000000000000000000000000000008E
:104230000000C000C000C000C000FF00FF00FF0081
:104240003000C300F300CF00FF00C300F300CF0035
:10425000FF00C300F300CF00FF00FF00FF00FF00DE
:104260000500FF00FF00FF00FF00FF00FF00FF0050
:10427000FF00FF00FF00FF00FF00FF00FF00FF0046
:10428000FF00FF00FF00FF00FF00FF00FF00FF0036
:10429000FF00FF00FF00FF00FF00FF00FF00FF0026
:1042A000FF00FF00FF00FF00FF00FF00FF00FF0016
:1042B000FF00FF00FF00FF00FF00FF00FF00FF0006
:1042C000FF00FF00FF00FF00FF00FF00FF00FF00F6
:1042D000FF00FF00FF00FF00FF00FF00FF00FF00E6
:1042E000BA00FF00FF00FF00FF00FF00FF00FF001B
:1042F000FF00FF00FF00FF00FF00FF00FF00AA001B
:00000001FF
